:020000040000FA
:06000000FE300C303A282E
:08000800A000030E8301A1001A
:100010000A08A2008A01AA1503140B190310003064
:100020008100A30DA40DA50DA90B1F282A162508D4
:10003000A8002408A7002308A6001930A9008B10E7
:100040000B1122088A00210E8300A00E200E090049
:0C007400203084008001840A80300402E7
:10008000031C3C281F30CE000130CA00CB0080305A
:10009000CD000E30F4003230D70083161F308505B6
:1000A000003086050B3087058312850186018701A4
:1000B000103083168E008312703083168F008312E7
:1000C0000030031799000313003003179A0003133D
:1000D0000C30970000309F00003083169F00831281
:1000E000183003179E000313003003179F000313FB
:1000F000803083168100831211309000043092000A
:100100007F308316920083120030950000308316F2
:100110009400831223309400A63083169800831233
:10012000003083169B00831210309800193083161C
:1001300099008312003083168C00831200308316DE
:100140008D00831200308B000D161924E91FAE2894
:1001500083160510851083120514851481018E0104
:100160008F010B118B100B108C018D010D168B174D
:100170001230E000FA215D2731177021D5220021CD
:10018000661A0721E61A02212A1A0C218F08031980
:10019000BE288F01E61A0717661A07157024B11BCF
:1001A0007F21661A0721E61A0221EE23DB233D2276
:1001B000B722E70BE628301EE128B20BE128301207
:1001C0005727401FE628E30BE6284013661A07214D
:1001D000E61A02214F18B921661A0721E61A0221F0
:1001E0004F18BE28AA19FA28CC0BBE28AA1AFE2836
:1001F0001930A900AA110C30CC00BE286821BE28F5
:10020000640008006B080E020318071308006B084F
:100210000E020318071108002A12C1302802031D1C
:100220001C292708BE002608BD0007303E0203191E
:100230007127BF2319246329280827062602031DD6
:100240000800F7302802031D28292708BF0063296A
:10025000A1302802031D2F292708F0006329A230AE
:100260002802031D36292708C2006329A730280267
:10027000031D47292A10A71B2A1427087F39EA00E3
:100280002A1CEA012B142A1C2B10AB156329C2303F
:100290002802031D63292708C40064000D1E4E298F
:1002A0008B13440803178D0083168C130C148312D0
:1002B0000C080313C5008B177F3044023730031935
:1002C000C500CE166329AA16AA110A30CC00080070
:1002D0004F144F150B1283160511831205150800D4
:1002E0004F10CF101930A900AA12AA110A30CC0061
:1002F0008316051583128B100B110B160800E81CD2
:10030000080034080319080034083702031D8E2939
:1003100035083802031D8E29B1130800AF0A0130D9
:100320002F02031D962934089300080007302F027E
:10033000031D9D293508930008000D302F02031D71
:10034000A7293608031908003608930008000E3064
:100350002F02031D08003408B7003508B800B401A7
:10036000B501B601AF01B113311F08006727311382
:1003700008004F19C629C9030F304905031D08009D
:10038000C9080319C6290515C90E080005114F1122
:10039000CF1870294B184608CB1847084B19480846
:1003A0004D05031DD6294430C900D9291130C90093
:1003B000D9290310CD0C0318DE2908008030CD00A8
:1003C0000310CB0DCB19E52908000130CB0010300C
:1003D000CE1ACA00410840028030031DCA00031033
:1003E000CA0D03184A144A084E050319E529FA21D3
:1003F000CF140800C601C701C8014A1C052A77307E
:10040000C6004008C700C100392ACA1C0C2A663041
:10041000C6004308C700392A4A1D132A5530C600B2
:100420007108C700392ACA1D1C2A4430C6005F085B
:10043000C700FF30DF00392A4A1E2F2A3330C6009A
:100440008B13343003178D0083168C130C14831216
:100450000C08031384008B170008C700392ACA1E32
:1004600008002130C6004408C7004508C800CE1265
:10047000080046084706C8000800051C452A401E1B
:10048000532AB90B532A4012532A401A532AB90A45
:100490003C083902031D532A4016691C532A3016A2
:1004A00057270530B200851C5B2AC01D692ABA0B8C
:1004B000692AC011692AC019692ABA0A3C083A0295
:1004C000031D692AC015E91C692A30165727053013
:1004D000B200851D712A401D7F2ABB0B7F2A401167
:1004E0007F2A40197F2ABB0A3C083B02031D7F2A52
:1004F0004015691D7F2A301657270530B20087192D
:10050000C010871DC0143F1886163F1C8612C219E2
:100510000224C2198F2A2A1B02242A1F0712E81953
:10052000962ABF1C8613BF1886179A2ABF1C8617E7
:10053000BF1886133F1F6613401CA12A3F1BA12A28
:10054000E617C01CAA2A681DAA2A71080319AA2A3C
:10055000F1017D23C318B32A2B1CB32A053077027F
:100560004310031C43146615C21E66110800B11B1C
:100570000800E008031D080031084206013903198C
:10058000C82A301342183017572731104218311437
:1005900031084206023903190800B110C218B1141B
:1005A000301657270530B2000800EA080319DF2A81
:1005B000AB18E72A6A0895002A18E12A0800950175
:1005C000080006162B14AB10421AAB1408002B1DA2
:1005D00008002B11D518322BD70B08003230D7006A
:1005E000D514AB1906238B131D3003178D0083160A
:1005F0008C130C1483120C080313DE006A08950098
:100600002A1C0800AB10421AAB140800AB112130B1
:10061000BF1C013E03178D0083168C130C1483122C
:100620000C080313D8008B17203003178D00831696
:100630008C130C1483120C080313DC008B1758085E
:100640005C07D9005C07DA005C07DB003030031779
:100650008D0083168C130C1483120C080313DD0019
:100660008B170800DE080319372BDE030800580833
:100670007702031C492B59087702031C4B2B5A089D
:100680007702031C4D2B5B087702031C4F2BD40A07
:10069000512BD00A512BD10A512BD20A512BD30AFC
:1006A000512B5008510452045304540410390319B7
:1006B0000800D601501AD614511A5615521AD615DA
:1006C000531A5616541AD616D001D101D201D301AD
:1006D000D401D5103230D7006A08ED005D075619F5
:1006E000ED005D07D619ED005D07561AED005D07B8
:1006F000D61AED006D08950008000030BE007108A4
:10070000BD00BF230800F10A720A71020318F1004C
:100710000800F103720AF11BF107080064000D1EC6
:100720008F2B8B13063003178D0083168C130C143C
:1007300083120C0803138B173F1D3030F200F203B5
:10074000701BBC2B700871020319BA2B0318B22B53
:100750000319B22B71087002BF187202BF18013E54
:10076000F300080070087102BF1C7202BF1C013E3A
:10077000F3000800F3010800FA30F30008000D123E
:100780003E08831203178D00831203133D08831262
:1007900003178C00831603178C130C158B138B1BFC
:1007A000CE2B55308D00AA308D008C148B170C1178
:1007B000831203130800F40BEB2B0E30F4009F148C
:1007C0007503F6009F18E22B2A151E08F5005F023C
:1007D00075080318DF008D309F0008009F149F18D4
:1007E000EF2B2B158B1383161E0883128B17F70024
:1007F0001E08C310031DC314FF30C318F7001130C7
:100800009F000800AD132D13AD0B0800AC0A033098
:100810002C02031C080007121E302E1C0A302C026A
:10082000031C0800AE0A0130E81AAE000716AC013E
:10083000080064000D1E1A2C8B13003003178D0066
:1008400083168C130C1483120C080313F1008B1302
:100850008B1B272C083003178D0083168C130C1468
:1008600083120C080313E8008B178B138B1B352C9A
:10087000093003178D0083168C130C1483120C0897
:100880000313E9008B171C3003178D0083168C139C
:100890000C1483120C080313BC008B170800070804
:1008A000403A870008000708043A87000800070854
:1008B000103A870008000608103A8600080006086B
:0E08C000203A860008000608803A86000800EC
:1008E000143060020318E00104308A0060088207B7
:1008F0008C2CA82C472D552D642D7D2DA72DBB2D7F
:10090000E92D232E5F2E8C2E9F2EAD2EBC2ED52EA4
:10091000EF2EFA2E052F0C2F071707112A1C06128F
:10092000FA01FB01EB01E6134010C012C313661B72
:1009300008003F1F0800421F66178E23F3080319A3
:100940000800421BE810421BE6170130E0000800D7
:10095000AB104014661DB01757272A17C311431355
:100960008B13053003178D0083168C130C14831220
:100970000C080313EC008B178B13033003178D0047
:1009800083168C130C1483120C080313F8008B17B6
:100990008B13043003178D0083168C130C148312F1
:1009A0000C080313F9008B178B130C3003178D0001
:1009B00083168C130C1483120C080313FC008B1782
:1009C0008B130D3003178D0083168C130C148312B8
:1009D0000C080313FE008B178B130F3003178D00C9
:1009E00083168C130C1483120C080313FD008B1751
:1009F0008B130E3003178D0083168C130C14831287
:100A00000C080313FF008B178B131B3003178D008B
:100A100083168C130C1483120C080313E4008B1739
:100A20008B13133003178D0083168C130C14831251
:100A30000C080313E5008B170130BF1C013E8B131C
:100A400003178D0083168C130C1483120C080313E8
:100A5000EF008B171130BF1C013E8B1303178D0065
:100A600083168C130C1483120C080313EE008B17DF
:100A7000421BEC010130421BE5006C08E100FF3035
:100A8000EB000230E000EC0803194E2D0800E616DA
:100A9000E10B08006C08E100EB0B0800E6126508AA
:100AA000E100E2010330E000080007130711E20B48
:100AB0000800E10B08006C08E100EB010430E000E5
:100AC000EC0803196C2D08006616E10B08006C0891
:100AD000E100EB0F0800EB0366128B1314300317D1
:100AE0008D0083168C130C1483120C080313E10081
:100AF0008B17E2010530E000080007130715E81C1A
:100B00008F2D66198F2DE10803198F2DE81F3016E0
:100B1000E81B30175727E20B0800E10B0800E81F1D
:100B20003012E81B301357278B13163003178D0034
:100B300083168C130C1483120C080313E1008B171B
:100B4000E2010130421BE1000630E0000800E20B48
:100B50000800E10B08008B13183003178D00831673
:100B60008C130C1483120C080313E1008B17E201A1
:100B70000730E0000800C0160616AB156E08EA0044
:100B8000AB14681CAB10E61444272B14E20B0800CE
:100B9000E10B08000130E61BF300AB1001307302DB
:100BA000031DD92D6E08EA00AB14681CAB10E610CB
:100BB00031278B13193003178D0083168C130C14F7
:100BC00083120C080313E1008B17E2010830E000E8
:100BD00008001427780875020318F32D7F08FB021C
:100BE000031CF82D08007F08FB070318122E0800CD
:100BF000FB010130E61BF300AB1001307302031D53
:100C0000082E6E08EA00AB14681CAB10E610312702
:100C1000E20B0800E10B0800C315F3012A131130A1
:100C2000E0000800FB018B131A3003178D008316B8
:100C30008C130C1483120C080313E1008B17E201D0
:100C40000930E0000800142779087502031C2D2ED6
:100C50007F08FB02031C322E08007F08FB070318E5
:100C60003C2E0800FB01E20B0800E10B08004317D3
:100C7000F3011130E0000800BF1C8323BF18892353
:100C8000F31B4F2EF30B4F2E6E08EA00AB14681CBB
:100C9000AB10E61031270A30E000FA0108008B1390
:100CA000193003178D0083168C130C1483120C0853
:100CB0000313E1008B17E2010830E00008002A1D51
:100CC00008002A1175087602031C6B2E7C08FA02B4
:100CD000031C722E08007E08BF1C7D08FA0703184B
:100CE000742E0800FA010800FA018712EA012B109D
:100CF000AB102B278B131730421B333003178D009B
:100D000083168C130C1483120C080313E1008B1749
:100D1000E2010B30E00008007D23C0120612E20B56
:100D20000800B0135727E10B0800EC080319A62EA2
:100D30006C08E100FF30EB000C30E00008006616A4
:100D4000E10B08006C08E100EB0B08006612650877
:100D5000E100E2010D30E000080007130711E20B8B
:100D60000800E10B08006C08E100EB010E30E00028
:100D7000EC080319C42E0800E616E10B08006C0805
:100D8000E100EB0F0800EB03E6128B13153003179D
:100D90008D0083168C130C1483120C080313E100CE
:100DA0008B17E2010F30E000080007170711E81C5D
:100DB000E72E6619E72EE1080319E72E681F3016A3
:100DC000681B30175727E20B0800E10B0800681F6B
:100DD0003012681B301357271030E00008002A1328
:100DE0002B270F30E3007108700203194017003001
:100DF000E00008002A132B27B0138712EA012B10FA
:100E0000AB1006120030E0000800C3171430E100F8
:100E1000E2011330E0000800C317E20B0800E10B09
:100E200008000030E0000800E61C0800E40B0800A1
:100E30008B131B3003178D0083168C130C14831235
:100E40000C080313E4008B17EA0A6F086A02031DFB
:100E50000800E61008002430B4000030B500B117D7
:100E600008002430B4008B131E3003178D00831646
:100E70008C130C1483120C080313B6008B178A15FD
:100E800012218A11B11708002430B4008B131F30CF
:100E900003178D0083168C130C1483120C08031394
:100EA000B6008B178A1512218A11B1170800063077
:100EB000B4003008B500B11708001430AF00FE30A0
:100EC000B400D930B500FF30B600B11708001430B7
:100ED000AF00FE30B400E530B500FF30B600B1170A
:100EE0000800B701FE30B400A130B5008A1500211A
:060EF0008A11B117080091
:10120000B6013D18B617BD1836173D19B616BD19EB
:1012100036163D1AB615BD1A36153D1BB614BD1B44
:1012200036140800B5013618B517B6183517361933
:10123000B516B6193516361AB515B61A3515361B44
:06124000B514B601080020
:084000000B00000003000700A3
:02400E00CC03E1
:1042000000007E007E00AA0096000A001800FF0051
:1042100087000000FF00FF0041002E0014002E0068
:1042200000003200320002001400150016003700B2
:104230000600190080005A00FF000A00010060001B
:10424000050040004000FF00FF00FF00FF00FF00EE
:10425000FF00FF00FF00FF00FF00FF00FF00FF0066
:104260000A00FF00FF0022007700FF00FF00FF00B0
:10427000FF00FF00FF00FF00FF00FF00FF00FF0046
:10428000FF00FF00FF00FF00FF00FF00FF00FF0036
:10429000FF00FF00FF00FF00FF00FF00FF00FF0026
:1042A000FF00FF00FF00FF00FF00FF00FF00FF0016
:1042B000FF00FF00FF00FF00FF00FF00FF00FF0006
:1042C000FF00FF00FF00FF00FF00FF00FF00FF00F6
:1042D000FF00FF00FF00FF00FF00FF00FF00FF00E6
:1042E000FF00FF00FF00FF00FF00FF00FF00FF00D6
:1042F000FF00FF00FF00FF00FF00FF00000037008D
:00000001FF
